:1000000008308A005E2900008A1D0A128A190A1621
:100010008A11831A0F28A500030EA6001428831244
:10002000A500030EA600A6140A08AD00A50E04083C
:10003000A7002008A8002108A9002208AA00230878
:10004000AB002408AC0083128B1E28280B1946280D
:100050008C308400001C2E280C18482827088400A7
:100060002808A0002908A1002A08A2002B08A30044
:100070002C08A4002D088A000A1A8A150A12260ED6
:1000800083008312250EA618831609008A114A28B8
:100090008A115228B60B4F28B50A0F30B6000B1143
:1000A0008A112E28B10A0319B20A0C108A112E28BF
:1000B000831685118312851113080230930083166D
:1000C0001418642883125F28831213086F089300A2
:1000D000831614186D288312682883121308700879
:1000E00093008316141876288312712885118312C1
:1000F000851500340F30EF009030F00058202A3082
:10010000EF00F00158202930EF00D030F0005820E7
:100110002830EF000230F00058203030EF0002307D
:10012000F00058204030EF000230F00058205030EE
:10013000EF000230F00058200D30EF00F0015820A1
:100140006030EF002030F00058202030EF00FF300A
:10015000F00058202130EF00E030F0005820EF018F
:100160004830F00058200130EF00F00158200430F2
:10017000EF00F00158200530EF00F00158207030FA
:10018000EF002230F00058202430EF00FF30F00064
:1001900058202530EF00E030F00058200830EF0004
:1001A0000230F00058200930EF00F00158200C30E8
:1001B000EF000F30F00058202B30EF00F0015820F6
:1001C0000F30EF00F00158203130EF000830F00020
:1001D00058203230EF00F00158203530EF00063063
:1001E000F00058204130EF000330F000582042303A
:1001F000EF00F00158204530EF000630F0005820A5
:100200005130EF000830F00058205230EF00F0017C
:1002100058205530EF000630F00058208A15732919
:1002200085118316851183121308A030930083165D
:1002300014181C298312172983121308930183169B
:100240001418242983121F2983121308EF0085151F
:100250008316851183126F08A1000034851183165F
:1002600085118312130803309300831614183A295A
:1002700083123529831213086F089300831614180C
:10028000432983123E2983121308930183161418FD
:100290004B298312462983121308F0008515831613
:1002A000851183127008A100003410212108ED008F
:1002B0006D1C92296630EF002E21A108031D6029D4
:1002C0006730EF002E212108EE006E08C03900389B
:1002D000031D92295130EF000830F00058205230B1
:1002E000EF00F00158205530EF000630F0005820A4
:1002F0003630EF006630F00058203730EF006E08DF
:10030000F00058203830EF00F00158203930EF006D
:10031000F00158203A30EF00F00158203B30EF0058
:10032000F00158202C30EF00F00158208A15A22946
:10033000851183168511831213088130930083166B
:100340001418A42983129F298312851583168511F9
:1003500083128A15302A8E30A0006E08A1006D0825
:10036000A200A301A108031DBF292208A100A20128
:100370000830A002A108031DBF29A001C72903104E
:10038000A11BC629A20DA10DA003BF29A113000026
:1003900000346D0803193A2AF500710803193A2A46
:1003A000F507031CD429DB297F30F502031C3A2A08
:1003B00003193A2ADF298130F50703183A2A75080C
:1003C000A000A101A201A3016E08F900F9176F08AE
:1003D000F8007008F7001830F500F601771C082ABD
:1003E0007408A307031CFA29A20A031DFA29A10A0B
:1003F0000319F6177308A207031C012AA10A03199F
:10040000F6177208EF00EF176F08A1070318F61729
:10041000F60DA10CA20CA30CF90CF80CF70C0310B0
:10042000F50BED290130A00703183A2AA11B1F2A5A
:10043000F90DA30DA20DA10DA00303193A2AF91F6E
:10044000302AA30A031D302AA20A031D302AA10A5A
:10045000031D302AA10CA20CA30CA00A03193A2AEE
:100460006E08F6007208F606F61F382AA1173E2A13
:10047000A1133E2AA001A101A201A30100008A1537
:10048000662B80300418F206F7016E08F600720839
:10049000F6066D080319302BF5007508A0007108E9
:1004A0000319392BF5020319D62A0318582A942A5E
:1004B0007208FB00FB177308FA007408F900F801D2
:1004C0000310FB0CFA0CF90CF80CF50B5F2AF61F65
:1004D0006C2A77144D2B77107510771670308400C6
:1004E000622B7712F61B7E2A751C892AFB0CFA0CEC
:1004F000F90CF80CA00A0319482B892AFB1B8C2A3B
:100500000310F80DF90DFA0DFB0DA0030319482B8C
:100510007E2A7717F52A77136E08F600F61F922ABF
:10052000FB17412BFB13412B7108F5007508A00048
:100530006D08F5026E08FB00FB176F08FA007008E3
:10054000F900F8010310FB0CFA0CF90CF80CF50B90
:10055000A12AF61FAE2AF7144D2BF7107510F716C7
:1005600074308400622BF712F61BC02A751CCB2A4C
:10057000FB0CFA0CF90CF80CA00A0319482BCB2A37
:10058000FB1BCE2A0310F80DF90DFA0DFB0DA0038D
:100590000319482BC02AF717F52AF7137208F6003B
:1005A000F61FD42AFB17412BFB13412B7208FB00CB
:1005B000FB177308FA007408F900F61FE32AFB130F
:1005C00077154D2B7711F801751070308400622B70
:1005D000F61B0B2B6E08F600751CF52AFB0CFA0CAB
:1005E000F90CF80CA00A0319482BF81F062BF90A7E
:1005F000031D062BFA0A031D062BFB0A031D062BFF
:10060000FB0CFA0CF90CA00A0319482B771B8B2A58
:10061000F71BCD2A2A2B8030FB06FB1F132B4D2BFB
:100620007208F600202B6E08F600FB08031D202B35
:10063000FA08031D202BF908031D202BA001412BD4
:10064000FB1B2A2B0310F80DF90DFA0DFB0DA00B67
:10065000202B482BF61F2E2BFB17412BFB13412B76
:100660007108A0007208FB007308FA007408F90012
:10067000412B6D08A0006E08FB006F08FA0070089F
:10068000F9007B08A1007A08A2007908A300812B59
:10069000A001A101A201A301812BF909FA09FB091B
:1006A000F809F80A031D5B2BF90A031D5B2BFA0AF4
:1006B000031D5B2BFB0A77186B2AF718AD2A7719F5
:1006C000E22A102B0008F907031C6C2BFA0A031D01
:1006D0006C2BFB0A0319751484030008FA07031C2A
:1006E000742BFB0A0319751484030008801B792BF3
:1006F000803AFB0703187514771A712AF71AB32A80
:10070000E82A00008A157A2B7008A1016F020318ED
:100710008C2B6F08A000982BA0010830F100EF0D82
:10072000A00D700820020318A000A10DF10B8F2B63
:1007300000346E18B42BEE18C82B6D08EF0064302F
:10074000F00084232008ED0021083030031DAD2B7C
:100750006E19B42BEE192030AF2B6E11EE11A107DC
:1007600021080C1EB12B99006D08EF000A30F00033
:1007700084232008ED0021083030031DC32B6E199F
:10078000C82BEE192030A10721080C1EC52B99009B
:100790003030ED076D080C1ECB2B990000348E30E5
:1007A000A0006D08A0026E08A2006F08A100A217A9
:1007B000A0080319E62B0310A208031DE22BA108D1
:1007C0000319E62BA20CA10CA00BDB2B00008A1551
:1007D000642C0408F600700EF038F200F207E23ED6
:1007E000F300323EF50070080F39F307F307F50701
:1007F000E93EF400F407F4076F0E0F39F407F5072C
:10080000F40DF50DF509F50D6F080F39F507F20D2B
:100810000730F1000A30F507F403031C0B2CF40732
:10082000F303031C0F2CF307F203031C132CF20732
:10083000F103031C172C76088400073084057130FF
:1008400084070008A000031D2B2C761A332CF61900
:100850002D2C20302E2C0830F6003030A007200838
:100860000C1E302C9900840A75300402031D212CC3
:100870000008A0003030A00720080C1E3D2C990075
:10088000003471080319072DFD0075080319072DA1
:10089000FD0203184C2C512C7F30FD070318072D47
:1008A000572C8130FD02031C072D0319072D7D08ED
:1008B000A000A101A201A301FC017208FB00FB172B
:1008C0007308FA007408F9001930FD007808F9027D
:1008D00003187A2C0130FA0203187A2CFB02031851
:1008E0007A2CFC0203187A2CFC0AFB0AFA0A780814
:1008F000F907AC2C7708FA020318952C0130FB029B
:100900000318952CFC020318952CFC0AFB0A7708A7
:10091000FA077808F907031CAC2CFA0A031DAC2C63
:10092000FB0A031DAC2CFC0AAC2C76088038FB02B9
:100930000318AB2C0130FC020318AB2CFC0A760820
:100940008038FB077708FA07031C892CFB0A031D74
:10095000892CFC0A892C2314FD0BAF2CBA2C031014
:10096000F90DFA0DFB0DFC0D0310A30DA20DA10D49
:10097000FE0D662C7E1CC22C0310A10CA20CA30C35
:10098000FE0CC52CA0030319072DFE1BEE2C031033
:10099000F90DFA0DFB0DFC0D7808F9020318DA2C9D
:1009A0000130FA020318DA2CFB020318DA2CFC02DD
:1009B000031CFD2C7708FA020318E52C0130FB021A
:1009C0000318E52CFC02031CFD2C76088038FB0282
:1009D0000318EE2C0130FC02031CFD2CA30A031D9E
:1009E000FD2CA20A031DFD2CA10A031DFD2CA00A4B
:1009F0000319072DA10CA20CA30C7208FD007608A8
:100A0000FD06FD1F052DA1170B2DA1130B2DA00118
:100A1000A101A201A3010000003404088316A5006F
:100A2000A6018312F61F182D2D300C1E152D9900CE
:100A3000F61775080319002E7F307502031CA22DCE
:100A4000F5008316AB010430AC0083120310F80DDF
:100A5000F70DF60D8316A60DAC0B2F2D312D83123D
:100A6000262D8312043075020318422D03307502BF
:100A7000031DF42D0A30831626020318412D83121C
:100A8000F42D83120330F5028316AB0A8312062776
:100A90000310F80DF70DF60D8316A60D8312DC2654
:100AA00002308316AC00831203108316A60C831247
:100AB000F60CF70CF80C8316AC0B5F2D612D83122E
:100AC000542D8312062704308316AC0083120310C2
:100AD0008316A70CA80CA90CAA0CAC0B702D722DB8
:100AE0008312672D8312DC26062783162908AA00A5
:100AF0002808A9002708A800A7018312DC260627DA
:100B000083162808AA002708A900A701A8018312B4
:100B1000DC268316A61D8E2D8312322D8312F50836
:100B2000031D992DF80AF70AF60A8316A60A8312FE
:100B3000F42D0310F80DF70DF60D8316A60D831294
:100B4000F503322DF509F50A7F30F5078316AB0161
:100B50000430AC0083120310F80DF70DF60D831668
:100B6000A60DAC0BB42DB62D8312AB2D0430831221
:100B7000F50705307502031C042E06270310F80D37
:100B8000F70DF60D8316A60D03108312F80DF70D61
:100B9000F60D8316A60D8312DC260310F80DF70D53
:100BA000F60D8316A60DAB0A0330AC0083120310BA
:100BB0008316A60C8312F60CF70CF80C8316AC0BFC
:100BC000E22DE42D8312D72D03308312F502831614
:100BD000261AEC2D8312B92D0310A60C8312F60CE5
:100BE000F70CF80CF503B92DF509F50A0330F507F4
:100BF00083162B08A100A300250AA3078312452E04
:100C00008316250AAB00831230300C1E052E990086
:100C10008316A508031D0E2E8312DA2E2E308312A2
:100C20000C1E102E990083162B08A400A40325087F
:100C3000240203181D2E8312202E2508A4008312DF
:100C40008316A408031D262E8312322E8312303001
:100C50000C1E282E99008316A40B2F2E312E8312E2
:100C6000272E831283162B08AC00250AAC02031C26
:100C70003B2E8312172F8312F5038316250AA30038
:100C80002B08A3022308A100831283162608A000C4
:100C9000831275080319582E8316A20083120310BD
:100CA0008316A00CA20B552E572E83124F2E8312A3
:100CB00083162308031D5E2E8312DA2E30302007A0
:100CC00083120C1E612E99008316210803196A2EC7
:100CD0008312742EA508031D6F2E8312DA2E2E3078
:100CE00083120C1E712E99008316A103A303031D0A
:100CF0007B2E8312DA2E8312750803198B2E83162E
:100D0000A200831203108316A00DA20B882E8A2E38
:100D10008312822E831283162008A6022608A700BB
:100D2000831276088316A800831277088316A90019
:100D3000831278088316AA0003108312F80DF70DAA
:100D4000F60D8316A60D03108312F80DF70DF60DA0
:100D50008316A60D2A088312F807031CB82EF70F76
:100D6000B82EF60AF608031DB82E8316A60A8312BB
:100D7000831629088312F707031CC52EF60AF60806
:100D8000031DC52E8316A60A831283162808831214
:100D9000F607031CCE2E8316A60A83128316270895
:100DA000A60703108312F80DF70DF60D8316A60D96
:100DB0008312452E0000172F83162A088312F80786
:100DC000031CEB2EF70FEB2EF60AF608031DEB2E95
:100DD0008316A60A8312831629088312F707031CB9
:100DE000F82EF60AF608031DF82E8316A60A8312BB
:100DF000831628088312F607031C012F8316A60A00
:100E0000831283162708A607831200348316260848
:100E1000A700831276088316A8008312770883162A
:100E2000A900831278088316AA00831200340000F8
:100E30000034FF3FFF3FFF3FFF3FFF3FFF3FFF3FCC
:100E4000FF3FFF3FFF3FFF3FFF3FFF3FFF3FFF3FB2
:100E5000FF3FFF3FFF3FFF3FFF3FFF3FFF3FFF3FA2
:100E6000FF3FFF3FFF3FFF3FFF3FFF3FFF3FFF3F92
:100E7000FF3FFF3FFF3FFF3FFF3FFF3FFF3FFF3F82
:100E8000FF3FFF3FFF3FFF3FFF3FFF3FFF3FFF3F72
:100E9000FF3FFF3FFF3FFF3FFF3FFF3FFF3FFF3F62
:100EA000FF3FFF3FFF3FFF3FFF3FFF3FFF3FFF3F52
:100EB000FF3FFF3FFF3FFF3FFF3FFF3FFF3FFF3F42
:100EC000FF3FFF3FFF3FFF3FFF3FFF3FFF3FFF3F32
:100ED000FF3FFF3FFF3FFF3FFF3FFF3FFF3FFF3F22
:100EE000FF3FFF3FFF3FFF3FFF3FFF3FFF3FFF3F12
:100EF000FF3FFF3FFF3FFF3FFF3FFF3FFF3FFF3F02
:100F0000FF3FFF3FFF3FFF3FFF3FFF3FFF3FFF3FF1
:100F1000FF3FFF3FFF3FFF3FFF3FFF3FFF3FFF3FE1
:100F2000FF3FFF3FFF3FFF3FFF3FFF3FFF3FFF3FD1
:100F3000FF3FFF3FFF3FFF3FFF3FFF3FFF3FFF3FC1
:100F4000FF3FFF3FFF3FFF3FFF3FFF3FFF3FFF3FB1
:100F5000FF3FFF3FFF3FFF3FFF3FFF3FFF3FFF3FA1
:100F6000FF3FFF3FFF3FFF3FFF3FFF3FFF3FFF3F91
:100F7000FF3FFF3FFF3FFF3FFF3FFF3FFF3FFF3F81
:100F8000FF3FFF3FFF3FFF3FFF3FFF3FFF3FFF3F71
:100F9000FF3FFF3FFF3FFF3FFF3FFF3FFF3FFF3F61
:100FA000FF3FFF3FFF3FFF3FFF3FFF3FFF3FFF3F51
:100FB000FF3FFF3FFF3FFF3FFF3FFF3FFF3FFF3F41
:100FC000FF3FFF3FFF3FFF3FFF3FFF3FFF3FFF3F31
:100FD000FF3FFF3FFF3FFF3FFF3FFF3FFF3FFF3F21
:100FE000FF3FFF3FFF3FFF3FFF3FFF3FFF3FFF3F11
:100FF000FF3FFF3FFF3FFF3FFF3FFF3FFF3FFF3F01
:101000000408F600F701EE1F09282D300C1E0628F3
:101010009900EE176D080319A9287F306D02031C93
:101020006828ED00FC010430FD000310F00DEF0D09
:10103000EE0DF70DFD0B152804306D02031828285E
:1010400003306D02031DA2280A307702031CA22878
:101050000330ED02FC0A52210310F00DEF0DEE0DEE
:10106000F70D39210230FD000310F70CEE0CEF0CE8
:10107000F00CFD0B342852210430FD000310F80C55
:10108000F90CFA0CFB0CFD0B3E28392152217A0891
:10109000FB007908FA007808F900F801392152219B
:1010A0007908FB007808FA00F801F9013921F719ED
:1010B0001C28ED08031D6128F00AEF0AEE0AF70A62
:1010C000A2280310F00DEF0DEE0DF70DED031C2817
:1010D000ED09ED0A7F30ED07FC010430FD0003103F
:1010E000F00DEF0DEE0DF70DFD0B6F280430ED0741
:1010F00005306D02031CB02852210310F00DEF0DD6
:10110000EE0DF70D0310F00DEF0DEE0DF70D39217B
:101110000310F00DEF0DEE0DF70DFC0A0330FD008E
:101120000310F70CEE0CEF0CF00CFD0B90280330C5
:10113000ED02771E78280310F70CEE0CEF0CF00C84
:10114000ED037828ED09ED0A0330ED072B30FD00A3
:10115000B328F701EE01EF01F001FD01FC01B32816
:10116000ED032D30FD00F2017708F1006D08031941
:10117000BE28F3000310F10CF30BBA287608F30035
:1011800072087302031C0B29303071070C1EC6282D
:101190009900F208031DD0282E300C1ECD2899008E
:1011A000F20A6D080319D928F3000310F10DF30BAF
:1011B000D5287108F7027708F8006E08F9006F0863
:1011C000FA007008FB000310F00DEF0DEE0DF70DA7
:1011D0000310F00DEF0DEE0DF70D7B08F007031C6B
:1011E000F728EF0FF728EE0AEE080319F70A7A0836
:1011F000EF07031CFF28EE0AEE080319F70A790827
:10120000EE070318F70A7808F7070310F00DEF0D43
:10121000EE0DF70DB428000045300C1E0D29990085
:101220007D08031916290C1E13299900F4017C0866
:10123000F5000A30F502031C2D29F40AF502031803
:101240001D29F507303074070C1E24299900303011
:1012500075070C1E292999003729F50730300C1E17
:101260002F299900303075070C1E34299900000091
:101270005B297B08F007031C4329EF0F4329EE0A83
:10128000EE080319F70A7A08EF07031C4B29EE0A48
:10129000EE080319F70A7908EE070318F70A780829
:1012A000F70700347708F8006E08F9006F08FA00B5
:1012B0007008FB00003400008A157F2D84011F3068
:1012C00083050C30831699002230980090308312E9
:1012D0009800640083168712071687113030831236
:1012E00094008A117A288A15B001AF01B201B101C8
:1012F0000F30B60081010730A000A01D87290730FC
:101300008101813084000008C0390F3880006400FA
:10131000813084000008C039200480008B1607301B
:1013200090008C3084000014C0308B04B50105148B
:10133000831605108312063035020318A4296400B1
:101340008A1155298A159B298E018F018A11102136
:101350008A152108CF0064004F1C7C2A6400663087
:10136000EF008A112E218A152108D100D108031D12
:10137000B92964006730EF008A112E218A152108EF
:10138000D0005008C0390038031DCE290B12B0011F
:10139000AF01B201B1018E018F010B16EE010E08F3
:1013A000ED00F0010F08EF006F08A3000001A0009E
:1013B00023086E04B00020086D04AF003630EF0043
:1013C0006630F0008A1158208A153830EF002F0857
:1013D000F0008A1158208A153008ED003930EF00EE
:1013E0006D08F0008A1158208A153A30EF00310854
:1013F000F0008A1158208A153208ED003B30EF00CA
:101400006D08F0008A1158208A155008C039A000D4
:1014100040302002031D0C2A3530EF000630F0006A
:101420008A1158208A155008033900380319262AD2
:1014300050080339A000013020020319262A500861
:101440000339A00002302002031D682A64003730EF
:10145000EF005008F0008A1158208A158A11982947
:101460008A15500803390038031D422A8616831650
:1014700086128312861183168611831286108316B4
:101480008610831250080339A00001302002031D8A
:10149000552A8612831686128312861583168611A4
:1014A0008312861083168610831250080339A00019
:1014B00002302002031D682A8612831686128312C8
:1014C0008611831686118312861483168610831262
:1014D0005008C039A00080302002031D762A0B126C
:1014E000B001AF01B201B1018E018F012C30EF00CC
:1014F000F0018A1158208A15CF1C8D2D640076309A
:10150000EF008A112E218A152108D1009030510256
:10151000031DE22A7730EF008A112E218A15210857
:10152000B7007830EF008A112E218A152108B80003
:101530007930EF008A112E218A152108B9007B30FD
:10154000EF008A112E218A15D4012108D3007A30A8
:10155000EF008A112E218A15EE012108ED005308B3
:10156000A30000016D07A10023080318013E6E07C8
:10157000A3002108ED002308EE008A11AB218A1593
:101580002008BA002108BB002208BC002308BD00C7
:101590007D30EF008A112E218A15D4012108D30055
:1015A0007C30EF008A112E218A15EE012108ED0012
:1015B0005308A30000016D07BE0023080318013E75
:1015C0006E07BF0091305102031D832B7830EF006E
:1015D0008A112E218A15D4012108D3007730EF001B
:1015E0008A112E218A15EE012108ED005308A3006F
:1015F00000016D07C00023080318013E6E07C100FB
:101600007A30EF008A112E218A15D4012108D300E7
:101610007930EF008A112E218A15EE012108ED00A4
:101620005308A30000016D07C20023080318013E00
:101630006E07C3007C30EF008A112E218A15D40179
:101640002108D3007B30EF008A112E218A15EE018C
:101650002108ED005308A30000016D07A100230835
:101660000318013E6E07A3002108ED002308EE00D9
:101670008A11AB218A152008C4002108C500220860
:10168000C6002308C7007D30EF008A112E218A157D
:10169000EE012108ED008A11AB218A152008D50042
:1016A0002108D6002208D7002308D8005508ED00ED
:1016B0005608EE005708EF005808F0008F30F10090
:1016C0000030F200F300F4008A11C9298A15840160
:1016D0004408ED004508EE004608EF004708F0001A
:1016E0002008F1002108F2002208F3002308F4008A
:1016F0008A11412A8A152008C4002108C500220841
:10170000C6002308C70092305102031D872D6400D4
:101710007730EF008A112E218A152108C800783011
:10172000EF008A112E218A152108C9007930EF00B7
:101730008A112E218A152108CA007A30EF008A11F9
:101740002E218A152108CB007B30EF008A112E2133
:101750008A152108CC007C30EF008A112E218A15D1
:101760002108CD003230D9003030DA004A08F03993
:10177000A000A00E0F30A0052008A00030302007E8
:10178000DB004A080F39A00030302007DC002F3082
:10179000DD004908F039A000A00E0F30A005200898
:1017A000A00030302007DE0049080F39A00030309B
:1017B0002007DF002F30E0004808F039A000A00E1D
:1017C0000F30A0052008A00030302007E1004808B5
:1017D0000F39A00030302007E2002C30E3004B0826
:1017E000F039A000A00E0F30A0052008A000303076
:1017F0002007E4004B080F39A00030302007E50037
:101800003A30E6004C08F039A000A00E0F30A005D9
:101810002008A00030302007E7004C080F39A00056
:1018200030302007E8003A30E9004D08F039A000D8
:10183000A00E0F30A0052008A00030302007EA00DD
:101840004D080F39A00030302007EB00EC01593073
:101850008400003000040319332C0C1E2D2C0008CA
:101860009900840A292C2C300C1E342C990037083E
:10187000ED000230EE008A1199238A152C300C1EDF
:101880003F2C99003808ED000230EE008A119923B0
:101890008A152C300C1E4A2C99003908ED00EE01F7
:1018A0008A1199238A1501303702FC3E0318632DF3
:1018B000043E8F2D3A08ED003B08EE003C08EF0097
:1018C0003D08F0008A11CF2B8A152208EE0021086E
:1018D000ED002C300C1E6A2C9900093084006E0833
:1018E000F0006D08EF008A11E9238A152E300C1ED6
:1018F000772C990030300C1E7B2C990030300C1E58
:101900007F2C99003F08EE003E08ED008A11AB21C4
:101910008A152008ED002108EE002208EF002308B8
:10192000F0006D08F1006E08F2006F08F300700817
:10193000F4008830F5007A30F6000030F700F80047
:101940008A1141248A152008F1002108F20022089A
:10195000F3002308F4002C300C1EAC2C990004304A
:1019600084007108F5007208F6007308F700740827
:10197000F8008A110D258A154108EE004008ED0097
:101980008A11AB218A152008ED002108EE002208FB
:10199000EF002308F0006D08F1006E08F2006F08F8
:1019A000F3007008F4008530F5004830F600003090
:1019B000F700F8008A1141248A152008F100210857
:1019C000F2002208F3002308F4002C300C1EE62C51
:1019D0009900043084007108F5007208F60073085D
:1019E000F7007408F8008A110D258A15632D3A084E
:1019F000F1003B08F2003C08F3003D08F40085309C
:101A0000F5004830F6000030F700F8008A11412454
:101A10008A152008ED002108EE002208EF002308B7
:101A2000F0002C300C1E122D9900023084006D083D
:101A3000F5006E08F6006F08F7007008F8008A11CC
:101A40000D258A153F08EE003E08ED008A11AB21F6
:101A50008A152008ED002108EE002208EF00230877
:101A6000F0002C300C1E322D9900043084006D08DB
:101A7000F5006E08F6006F08F7007008F8008A118C
:101A80000D258A154108EE004008ED008A11AB21B2
:101A90008A152008ED002108EE002208EF00230837
:101AA000F0002C300C1E522D9900043084006D087B
:101AB000F5006E08F6006F08F7007008F8008A114C
:101AC0000D258A15632D2C300C1E642D99000930CC
:101AD00084004308F0004208EF008A11E9238A15C8
:101AE0002C300C1E712D9900043084004408ED0048
:101AF0004508EE004608EF004708F00000280A30CD
:101B00000C1E802D99000D300C1E842D99002C3058
:101B1000EF00F0018A1158208A15A62963000A14E3
:0E1B20008A100A1582075A2C5A2CF72C5A2CC0
:02400E00FA3F77
:00000001FF
